:0200000480007A
:100000006F004005732F2034930F8000630AFF03B5
:10001000930F90006306FF03930FB0006302FF038A
:10002000170F0000130F4F4E63040F0067000F00FF
:10003000732F203463540F006F00400093E19153FD
:10004000171F000023203FFC171F0000232E0FFA6C
:100050006FF01FFF930000001301000093010000E8
:10006000130200009302000013030000930300003A
:100070001304000093040000130500009305000022
:10008000130600009306000013070000930700000A
:1000900013080000930800001309000093090000F2
:1000A000130A0000930A0000130B0000930B0000DA
:1000B000130C0000930C0000130D0000930D0000C2
:1000C000130E0000930E0000130F0000930F0000AA
:1000D000732540F16310050097020000938202012E
:1000E000739052307350447497020000938202015F
:1000F00073905230735000189702000093824202AE
:10010000739052309B021000939252039382F2FF3D
:100110007390023B9302F0017390023A73504030A7
:100120009702000093824201739052307350203046
:100130007350303093010000970200009382C2ECAC
:1001400073905230130510001315F501635C050020
:100150000F00F00F930110009308D0051305000065
:100160007300000093020000638A02007390521033
:10017000B7B200009B82921073902230735000300F
:10018000372500001B05058073200530970200000D
:100190009382420173901234732540F17300203032
:1001A00093012000972000009380C0E53781400034
:1001B0001B01110C1311110113013128131111012D
:1001C00013018170970700009387470123B0200037
:1001D00003B700006F00800013070100B7834000E1
:1001E0009B83130C939313019383332893931301ED
:1001F000938383706310772E930130009720000063
:10020000938040E037A190001B01110B1311C10036
:100210001301D1C01311C1001301110E1311C1003C
:10022000130101F19707000093874701A3B0200055
:1002300003B710006F00800013070100B7A3900000
:100240009B83130B9393C3009383D3C09393C300F7
:100250009383130E9393C300938303F1631C772658
:1002600093014000972000009380C0D937211101ED
:100270001B0111131311C100130151411311C100CE
:10028000130111161311C1001301817197070000AA
:100290009387470123B1200003B720006F0080003F
:1002A00013070100B72311019B8313139393C3001A
:1002B000938353419393C300938313169393C30083
:1002C0009383837163187720930150009720000077
:1002D000938040D337D1C8001B01910D1311C10089
:1002E0001301F1E01311C1001301118F1311D1009B
:1002F000130101F29707000093874701A3B1200083
:1003000003B730006F00800013070100B7D3C800A7
:100310009B83930D9393C3009383F3E09393C30064
:100320009383138F9393D300938303F26314771A09
:1003300093016000972000009380C0CC3711090121
:100340001B0191111311C100130131211311C100BF
:10035000130111931311D10013018172970700004B
:100360009387470123B2200003B740006F0080004D
:1003700013070100B71309019B8393119393C300E3
:10038000938333219393C300938313939393D30065
:100390009383837263107714930170009720000099
:1003A000938040C637A192021B01312B1311C1006B
:1003B0001301D1C21311C1001301312E1311C10059
:1003C000130101F39707000093874701A3B22000B0
:1003D00003B750006F00800013070100B7A392021B
:1003E0009B83332B9393C3009383D3C29393C30014
:1003F0009383332E9393C300938303F3631C770C8F
:1004000093018000972000009380C0BF3721130321
:100410001B0131331311C100130151431311C100EA
:10042000130131361311C1001301817397070000C6
:100430009387470123B3200003B760006F0080005B
:1004400013070100B72313039B8333339393C30034
:10045000938353439393C300938333369393C3009F
:1004600093838373631877069301900097200000AD
:10047000938040B937F1E4001B01D18E1311C10004
:100480001301F1F01311C1001301914F1311E10099
:10049000130101F49707000093874701A3B32000DD
:1004A00003B770006F00800013070100B7F3E4008A
:1004B0009B83D38E9393C3009383F3F09393C300F2
:1004C0009383934F9393E300938303F46314770030
:1004D000631030020F00F00F638001009391110050
:1004E00093E111009308D00513850100730000000B
:1004F0000F00F00F930110009308D00513050000C2
:10050000730000009302600073232034E39462FCC4
:100510007390173473002030731000C00000000087
:1005200000000000000000000000000000000000CB
:1005300000000000000000000000000000000000BB
:1010000000000000000000000000000000000000E0
:1010100000000000000000000000000000000000D0
:1010200000000000000000000000000000000000C0
:1010300000000000000000000000000000000000B0
:081040000000000000000000A8
:1020000000000000000000000000000000000000D0
:040000058000000077
:00000001FF
